:100000000C942A001895000018950000189500001F
:10001000189500001895000018950000189500002C
:10002000189500001895000018950000189500001C
:10003000189500001895000018950000189500000C
:1000400018950000189500001895000018950000FC
:10005000189500008FE58DBFC0E0E2E84E2E88E0E5
:100060008EBFD8E0F7E05F2EEEEFF7E0A0E6B0E05D
:1000700088278D933197E9F785E089B980E080BDC5
:1000800088E18AB9662486E086B98C9A8D9A8E9A20
:100090008A9A8B9A379A5A924A9284E190E0A42DD8
:1000A000B52D8D939C9382E00E94E4025A924A926D
:1000B00081E0A42DB52D8C9381E00E94E4020E9482
:1000C0004502249683E00E94E0025A924A9284E11B
:1000D00090E0A42DB52D8D939C9382E00E94E402C4
:1000E0005A924A9282E0A42DB52D8C9381E00E9411
:1000F000E4020E944502249683E00E94E0025A92A4
:100100004A9284E190E0A42DB52D8D939C9382E0DA
:100110000E94E4025A924A9284E0A42DB52D8C9359
:1001200081E00E94E4020E944502249683E00E943E
:10013000E00281E08093AC0080E08093AB000E94FD
:100140007602969895989498EF93FF93E1E1F1E009
:100150000E942603FF91EF9181E08093600000915F
:1001600060000A3018F011F00C94C0000E94910257
:10017000A0E6B0E08C918F5F8C9310F40C94AF00EC
:1001800001EC16E12CE631E0A3E7B0E00D931D93FE
:100190002D933C938D9A8C9A9498A3E7B0E090E2CB
:1001A0008D91983018F4392F992702C038E0985073
:1001B0008795959808F4959A00000000949AEF931B
:1001C000FF93E2E0F0E00E942603FF91EF91949804
:1001D000EF93FF93E2E0F0E00E942603FF91EF919E
:1001E0003A9531F79923E1F68D9A8C9A9498ACEA76
:1001F000B0E098E08D91983018F4392F992702C01B
:1002000038E098508795959808F4959A000000007A
:10021000949AEF93FF93E2E0F0E00E942603FF91AF
:10022000EF919498EF93FF93E2E0F0E00E942603B1
:10023000FF91EF913A9531F79923E1F6969A0000F4
:1002400000000000000096980000000082B394E0D7
:10025000892782BB0E949103A7E8B0E03FE00E949B
:1002600000030E948E0341E050E060E070E0A7E8E8
:10027000B0E00E945F03A0E1B0E00D911D912D91CF
:100280003C910E944C0311F00C94490193980C94FA
:100290004A01939A0E949103A7E7B0E03FE00E94D1
:1002A00000030E948E030E949103A1EBB0E03FE0A7
:1002B0000E9400030E948E030E949103ABE9B0E00C
:1002C0003FE00E9400030E948E0300000000000037
:1002D0000000000000000000A7E7B0E00E945F03FC
:1002E000A3E7B0E00D931D932D933D93A1EBB0E0F8
:1002F0000E945F03ADEAB0E00D931D932D933D93F3
:10030000ABE9B0E00E945F03A7E9B0E00D931D9355
:100310002D933D9301E010E020E030E0AFE6B0E047
:100320000D931D932D933C93ADEAB0E04D915D91FB
:100330006D917C91AFE6B0E00D911D912D913C91B6
:100340000E944C031CF011F00C944302A3E7B0E0B0
:100350000D911D912D913C91A7E9B0E04D915D91DA
:100360006D917C910E944703A3E7B0E00D931D932C
:100370002D933D938D9A8C9A9498A3E7B0E090E2E8
:100380008D91983018F4392F992702C038E0985091
:100390008795959808F4959A00000000949AEF9339
:1003A000FF93E2E0F0E00E942603FF91EF91949822
:1003B000EF93FF93E2E0F0E00E942603FF91EF91BC
:1003C0003A9531F79923E1F68D9A8C9A9498ACEA94
:1003D000B0E098E08D91983018F4392F992702C039
:1003E00038E098508795959808F4959A0000000099
:1003F000949AEF93FF93E2E0F0E00E942603FF91CE
:10040000EF919498EF93FF93E2E0F0E00E942603CF
:10041000FF91EF913A9531F79923E1F6969A000012
:1004200000000000000096980000EF93FF93E1E1C8
:10043000F1E00E942603FF91EF9187E087B90E94C7
:100440003E03A1E6B0E08D939C9386E087B90E94BD
:100450003E03A3E6B0E08D939C93000000000000F3
:1004600032E0A1E6B0E00E941D03000000000000A1
:1004700032E0A3E6B0E00E941D03AFE6B0E00E94C8
:10048000E8020C9494010C94260181E090E0AAE625
:10049000B0E08D939C93AA81BB814D915C91AAE6BB
:1004A000B0E00D911C910417150718F011F00C9491
:1004B000740282B394E0892782BBA881B9818C91B0
:1004C00099270E942F0382B394E0892782BBA881D9
:1004D000B9818C9199270E942F03AAE6B0E00E946F
:1004E000F70210F40C944B0292980895939A82E3C9
:1004F00090E00E942F03939882E390E00E942F03E4
:10050000939A82E390E00E942F03939882E390E015
:100510000E942F03939A939882E390E00E942F0306
:10052000089500E010E020E030E0A5E6B0E00D9393
:100530001D932D933C938D9A8C9A9498A5E6B0E0E8
:1005400090E28D91983018F4392F992702C038E045
:1005500098508795959808F4959A00000000949A11
:10056000000000009498000000003A9591F799234C
:1005700041F780E0809369008D9A8C9A9498A9E65F
:10058000B0E098E08D91983018F4392F992702C087
:1005900038E098508795959808F4959A00000000E7
:1005A000949A000000009498000000003A9591F79A
:1005B000992341F7969A000096980895F894FFCFF2
:1005C000481A8827580A0895480E8827581E089503
:1005D0000D911D912D913C9181E0080F8827181FE6
:1005E000281F381F3C932E931E930E930895ED9170
:1005F000FC91EF5FFF4FFC93EE930895AAE6B7E0FE
:1006000018D0883091F08D3039F03323C9F38D93B1
:100610003A9563FE17D0F4CF63FC04C08DE012D08E
:100620008AE010D088278C9308950CD011973395C9
:10063000E7CF5F9BFECF8CB108958D9103D03A95A3
:10064000E1F708955D9BFECF8CB908953197F1F7DE
:100650000895689462F80895E89462F80895EF9315
:10066000FF93EE27E82BE92B31F0EDECFAE0319720
:10067000F1F70197D1F7FF91EF910895369A3699E6
:10068000FECF369A3699FECF84B195B10895040F06
:10069000151F261F371F089504171507260737074C
:1006A0000895000F111F221F331F08950095109504
:1006B000209530950F5F1F4F2F4F3F4F0895002714
:1006C0001127222733271DD08A3328F4803318F0CE
:1006D00005D015D0F9CF0EF4E9CF089580538F934C
:1006E000402F512F622F732FDCDFDBDFD0DFD9DF0C
:1006F0008F919927080F191F291F391F08958D9170
:100700000895E894FCDF8032E9F38B32D9F3893025
:10071000C9F38D3211F46894F2CF0895E89463F828
:080720000895689463F8089540
:00000001FF
